:02000000040AF0
:080008009F0C0200210A0E0CFE
:100010003000F90C27000000E7020B0AF002090A81
:100020000008050C2900F90C27000000E702150A5A
:10003000E902130A0008F90C27000000E7021D0A74
:100040000008080C0600080C2600050C2800010C0E
:1000500026000709010C26001109010C26001B09C6
:10006000E802270A050C2800020C26000709030CE9
:1000700026001109030C26001B09E802340A050CAE
:100080002800040C26000709060C26001109070C9D
:1000900026001B09E802410A050C2800100C260066
:1000A0000709140C26001109160C26001B09E8028A
:1000B0004E0A050C2800200C26000709300C2600EB
:1000C0001109340C26001B09E8025B0A050C280004
:1000D000200C26000709200C26001109300C2600F0
:1000E0001B09E802680A050C2800200C26000709F5
:1000F000200C26001109200C26001B09E802750AB5
:10010000050C2800100C26000709300C26001109E8
:10011000300C26001B09E802820A050C2800040C9A
:1001200026000709140C26001109340C26001B09AF
:10013000E8028F0A050C2800020C26000709060CAD
:1001400026001109160C26001B09E8029C0A050C62
:100150002800010C26000709030C26001109070CD2
:1001600026001B09E802A90A050C2800010C26003C
:100170000709010C26001109030C26001B09E802DF
:04018000B60A250A8C
:021FFE00EA0FE8
:00000001FF
